:100000000F0A050C2900E902030A0000000000089D
:10001000620C2900E9020A0A00000000000804003E
:1000200064000C0C2500F30C0500FF0C060000001A
:1000300065046505040005071A0A000001090602A7
:100040002700FC0E2800280328032707280A3D0A5A
:1000500007072B0A340A000045040809E8022E0AA3
:100060004505650465051A0A45040809E802360ACB
:1000700000004505650465051A0A0000000000003F
:1000800045040809E802420A00000000450565042D
:0400900065051A0ADE
:021FFE000E00D3
:00000001FF
